:030000000219FDE5
:03000B000200A848
:03002B0002015B74
:03005B000202E6B8
:030073000202D3B3
:1000800002030406080C10182030406080040608A3
:100090000C10182030406080A0C00003070F1F051F
:1000A000050D050305030302C2AFC0D0C0E0206206
:1000B00014E5256009E473E525F4F58AD262D0E001
:1000C000D0D0D2AF3285268AC262E526F4603030C5
:1000D000682620720DD0E0D0D0C290C291C292D2D8
:1000E000AF32C290C291C292206F0D20650A740196
:1000F000D5E0FDE57BF45290D0E0D0D0D2AF3275A0
:100100008A00C28DD26201F801B73068052065020D
:10011000D29001B7306805206502D29101B73068EE
:1001200005206502D29201B7D29330680A20650794
:100130007405D5E0FDD29001B7D29430680A2065ED
:10014000077405D5E0FDD29101B7D29530680A2039
:1001500065077405D5E0FDD29201B7C2AFC2AD53B9
:10016000E6EFC0D0C0E0D2D3D2AFC2CEE52A60075E
:10017000207449152A21BC7800790020742EE5806E
:10018000307E01F430E70278FF53DACF207E03435C
:10019000DA20307E0343DA10C2D8C271E580307EA7
:1001A00001F430E70279FFC3E89970CB3061037541
:1001B0002A18207403752A18885CD27020740DE503
:1001C0002B6004152B21CC43DA01C2D820700241E8
:1001D0003FA85C206102C270207431C3E894F040F3
:1001E0000374F0F8E8C4540F28F87984B703024187
:1001F0000CC313C3138721200802C313200A06C3AC
:10020000C898F8410C28F8500374FFF8C3E89565C6
:100210005003E565F88822E52D54066022206B1F07
:10022000E536C333C333F8E564C313C313F9C39589
:100230002240028922E82522F52250037522FF85FB
:100240002224A824C3E52495614002A8618825E5FD
:100250006670024183C3E8AA669A5003E8FAE4F99B
:10026000EAC333FBE568F45B29400D2567F8E567D1
:1002700060021567400B41830AC3E5679A50020587
:100280006778FF8826C26FC3E52694F84002D26FD4
:1002900020CF0AD0E0D0D043E610D2AD32C2CF0595
:1002A0003A7801E52A6005307402152AC3E55C94AA
:1002B000014005755F0041C9756000756900E55F23
:1002C0002401F55F5003755FFFD0E0D0D043E61006
:1002D000D2AD32C2AF53E67F7592FA7593FFC2601A
:1002E000759104D2AF32C2AF53E6EFC2ADC0D0C0F9
:1002F000E0C0F0D2D3D2AFA8FBA9FCC2D8307102C3
:10030000614D53DACF207E0343DA10307E0343DAA7
:1003100020D271E580307E01F420E7026124882735
:100320008928A17A53DACF207E0343DA20307E0376
:1003300043DA10C2D8C271307402A1667800E58039
:10034000307E01F430E702A166885CA14E53DACF1B
:10035000207E0343DA20307E0343DA10C27120612D
:1003600002812653DACF207E0343DA10307E034326
:10037000DA20C2D8D27188578958C3E89555F8E970
:100380009556F97B007E087A00C3E8948CE99400C6
:100390005005755B008118882178A2E6A821605578
:1003A000C3E894C8E994005008E4D2E4FB7A0A61F7
:1003B000F3C3E89468E994015008E4D2E3FB7A0FB0
:1003C00061F3C3E894D0E994025008E4D2E2FB7AE6
:1003D0001E61F3C3E894A0E994055008E4D2E1FB60
:1003E0007A3C61F3C3E89498E994085008E4D2E0B9
:1003F000FB7A787E00C3E89559FCE9955AFD30E711
:100400000AECF42401FCEDF43400FD755B00C3EC50
:100410009AED9E5003755B018859895A8557558519
:1004200058567802A14EC3E89527F8E99528F93087
:100430007C02A132307B02A132307A02A12B2075DE
:10044000028149E9FDE8FC8168E9C313F9E813F882
:10045000307902A12BE9C313F9E813F8307802A12F
:100460002BE9C313FDE813FC20612CC3EC941CEDB5
:0F04700094024002817FED701EC3EC94C85018B7
:10047F000529E52970021529C3E529940A5002A11F
:10048F0066755C00D270A166E5296002152978882F
:10049F00E6F97400207F087896B90302789EE62467
:1004AF00FAFEE43400FFC3EC9EFCED9FFD9208B909
:1004BF000310A2085007207609D27681D130760238
:1004CF00C276A2085016B9030DECF42401FCEDF42A
:1004DF003400FD0204EB78007900A132B90315EC6A
:1004EF0033FCED33FDC3EC940AFCED9400FD500496
:1004FF007C007D00C3EC94FFED9400400678FF79FB
:10050F0000A132EC8572F0A4C5F0A2F733F87900A0
:10051F00400302054E78FF790002054EE9C313F937
:10052F00E813F8307C0EE9600278FFC3E81338F85F
:10053F00E43400F9C3E894FFE99400400278FF889F
:10054F005CD270206102A166741FF4552F4BF52FFA
:10055F00C274EB7002D274752A18307403752A0AAC
:10056F00306102A17A20740353DAFE207403752BD5
:10057F0006D0F0D0E0D0D0D2AD43E61032790102F0
:10058F0005AA79030205AA790A0205AA791E0205AE
:10059F00AA79640205AA79C80205AA7817E4D5E0FA
:1005AF00FDD8FAD9F6227A147B780205D17A107B1E
:1005BF008C0205D17A0D7BB40205D17A0B7BC80270
:1005CF0005D1E573D5E001227902E4D294D5E0FD9F
:1005DF00D291D5E0FDC291D5E0FDC294D5E0FDE901
:1005EF0020E002D29030E002D292E573D5E0FDE92F
:1005FF0020E002C29030E002C2927496D5E0FDD99D
:10060F00C9EAF8D5E0FDD8FBDBB8D29422C37C0051
:10061F007D0075F00005F0EA33FAEB33FB50F6EB93
:10062F0013FBEA13FAC3E9FFE8FEE89AF8E99BF92E
:10063F005004EFF9EEF8B3EC33FCED33FDD5F0DFFA
:10064F00EDF9ECF822E889F08A20D2D4F8A9F07BF2
:10065F000030F70B7BFFF42401F8E9F43400F9E8DC
:10066F008520F0A4ADF0F8E98520F0A4AFF0FEED01
:10067F002EF974003FFA7C04C3EA13FAE913F9E880
:10068F0013F8DCF48BF030F70AE8F42401F8E9F4FE
:10069F003400F9E889F0C2D4F8A9F02222C3E54169
:1006AF0013F9E54013F8C3E54498F8E54599F95077
:1006BF000CC3E89480E994FF40160206E3C3E89464
:1006CF007FE9940050030206E3787F79000206E386
:1006DF00788079FF8849894A22E5492546F8E54A15
:1006EF003547F9854A20E4300701F43548FA30E7F9
:1006FF0009C3EA94F04015020721C3EA940F50038F
:10070F0002072178FF79FF7A0F020721780079001D
:10071F007AF0C3E5249561500AC374019524500BF8
:10072F0002073FE54A20E70E02073FE54A30E7069A
:10073F00884689478A482278A5E6FAC3E54933F8FF
:10074F00E54A33F9D154E930E70BC3E89480E994D3
:10075F00FF4013E179C3E8947FE994005002E179F7
:10076F00787F7900E179788079FFE820E715C3E594
:10077F002398F84009C3E8940140030207A07801C9
:10078F000207A0E8F424012523F840030207A0780C
:10079F00FF884B2278A6E6FAA847A948D154E9303A
:1007AF00E70CC3E89401E994FF40160207D4C3E8AD
:1007BF0094FFE9940050030207D478FF79000207F1
:1007CF00D4780179FFE920E715C3E54B98F8400984
:1007DF00C3E8940140030207FB78010207FBE8F42A
:1007EF002401254BF840030207FB78FF8824227869
:1007FF00FF20692879A1E76023E541601F74FF8519
:10080F0041F0848539F0306A0375F005A4F8C5F01E
:10081F00600278FFC3E895645002A864886322C31E
:10082F00E5409440E5419401E563500314013F0412
:10083F006002F563220208472275E890227883E66A
:10084F00FF30EDF9A8BDA9BE0570C3E5709408404F
:10085F0052757000E9FA79A0E76044EA7007E57114
:0F086F00601B020880C3E895716010E5715006A8
:10087E00600C1402088C0460F902088CE571F571A5
:10088E00C394F6401B7561C0C39406401375618016
:10089E00C39406400B756140C39406400375610016
:1008AE0075BB0622E561F460020561E570B40703CD
:1008BE0075BB1022743279A787F0A4C5F0A2F73366
:1008CE00F8C3E895614002A86188228824882588AB
:1008DE00268864227540007541F022C2AF75C8208B
:1008EE00A8CCA9CDAA3A30CF010A75C824D2AFAB95
:1008FE003BAC3C883B893CC3E89BF8E99C206908EB
:10090E00F930660221F82152AD3D8A3DF9EA9DFA91
:10091E00600478FF79FFAE3EAF3F8B3E8C3FA83B25
:10092E00A93CC3E89EF8E99FF9C3E54113FBE540F6
:10093E0013FAE82AF540E93BF54150067540FF757C
:10094E0041FF219FAA40AB41AC40AD417E047F02E6
:10095E00C3EB9404400D1E1FC3EB94084005206AA0
:10096E00021E1FC3ED13FDEC13FCDEF7C3EA9CFA67
:10097E00EB9DFBEF6009C3E913F9E813F8DFF7EA23
:10098E0028FAEB39FB8A408B4150067BFF8B408B5C
:10099E0041C3EB94025002D2663069047F0321CA30
:1009AE007892E6FFC3E537948240110FC3E5379482
:1009BE00A040010FC3EF940640027F057E02E54181
:1009CE00C4540FF9E541C454F0F8E540C4540F285F
:1009DE00F8C3E89EFAE99400FB4009C3EA9402EBDF
:1009EE00940050047A02E4FB4144AA40AB41EBC4AC
:1009FE00FEEAC4540F4EFCC3EA9CFAEB9400FBC310
:100A0E00E813C313F8EA28FAEB3400FB8A408B4153
:100A1E00C3EB94024002C2667802EBC4FE7B00EA8E
:100A2E00C4540F4EFAC3EA98FA4005C3940250021A
:100A3E007A027892E6FF30600241448551928552E7
:100A4E0093D26043E680C3E49AF8E49BF9306602E1
:100A5E0041D0E8FAE9FBD3E913FDE813FC8851898C
:100A6E0052C3EF94036038EF20E00DE82CF8E93D17
:100A7E00F9ECFAEDFB020A99E828F8E939F9C3E82E
:100A8E002402F8E93400F97AFE7BFFC3EF940340A9
:100A9E000E8A538B54884D894E8C4F8D506104882D
:100AAE005389548A4D8B4E8C4F8D5030691275532D
:100ABE00F07554FF754FF07550FF7551F07552FF7C
:100ACE006104E8FAD3E813FC8851C3EF9403602065
:100ADE00EF20E007E82CF8ECFA41F0E8282402F8C1
:100AEE007AFEC3EF940340088A53884D8C4F6104FD
:100AFE0088538A4D8C4FE568C3335002646BF5689A
:100B0E00306002610E753402D26043E680E52D54EA
:100B1E00066034A840A941C3E913F9E813F8C3E904
:100B2E0013F9E813F8306904E92440F9C2AF53E62B
:100B3E007F759100C3E498F594E499F59575910449
:100B4E00D26043E680D2AF22D26475430075200096
:100B5E00306C03752040020B75D26475430075200E
:100B6E0040306C0375200078017901206620E52D58
:100B7E0054066002C2647914E541C313700104F88F
:100B8E00C3941440027814306904781B791B2060DA
:100B9E0010E543600C306903D53404D26D812071A9
:100BAE00160543E59BF45440B52002810A306909CD
:100BBE0008C3E899400118619C20640A08C3E899AB
:100BCE0040026175619CC264C2AF53E67F759100AD
:100BDE003066127594007595F8759104D26043E6EF
:100BEE0080D2AF6175E5417EFFC3334005C333400C
:100BFE0001FEC3E49E759400F59561E7C3E5339459
:100C0E0001500261753064026175D802811E619CCB
:100C1E00C26DC2AF53E67F7591008553948554958E
:100C2E00759104854D92854E93D26043E680D2AF86
:100C3E00E52D54066008206A020533020C5C306D07
:100C4E000D206C0A2064071581158102151F22786C
:100C5E00003064027801E53775F007A4F9E5F02855
:0F0C6E00F5F0E9A2F013A2F113A2F213F537C3C8
:100C7D0094785003753778C3E53795384008D265B9
:100C8D00C290C291C2923060028193854F9285507D
:100C9D0093D26043E68022207D16C2AF754202D208
:100CAD0094C293306202D292D2AF759F11020E930D
:100CBD00C2AF754202D294C295306202D290D2AFC9
:100CCD00759F11020E93307243207D20C2AF754285
:100CDD0003900139757B10C292D295306204D29186
:100CED0081F1C294D2AF759F01020E93C2AF7542CE
:100CFD0003900139757B10C290D293306204D2916A
:100D0D00A111C294D2AF759F21020E93207D17C2FF
:100D1D00AF754203900114C292306202D291D2AFEC
:100D2D00759F01020E93C2AF754203900114C290DC
:100D3D00306202D291D2AF759F21020E93207D16A3
:100D4D00C2AF754204D293C295306202D291D2AF36
:100D5D00759F21020E93C2AF754204D295C2933096
:100D6D006202D291D2AF759F01020E933072432071
:100D7D007D20C2AF754205900128757B08C291D2C6
:100D8D0094306204D290A197C293D2AF759F110295
:100D9D000E93C2AF75420590014A757B20C291D268
:100DAD0094306204D292A1B7C295D2AF759F110251
:100DBD000E93207D17C2AF75420590010AC2913086
:100DCD006202D290D2AF759F11020E93C2AF7542DF
:100DDD000590011EC2913062EBD292D2AF759F1178
:100DED00020E93207D16C2AF754206D295C2943085
:100DFD006202D290D2AF759F01020E93C2AF7542BF
:100E0D0006D293C294306202D292D2AF759F210264
:100E1D000E93307243207D20C2AF75420190014A7E
:100E2D00757B20C290D293306204D292C13DC2959F
:100E3D00D2AF759F21020E93C2AF7542019001286A
:100E4D00757B08C292D295306204D290C15DC29377
:100E5D00D2AF759F01020E93207D17C2AF7542016F
:100E6D0090011EC290306202D292D2AF759F2102C4
:100E7D000E93C2AF75420190010AC292306202D246
:100E8D0090D2AF759F01C26522900108757B00C29B
:100E9D0090C291C292D293D294D295C2622278809E
:100EAD0076FF0876FF0876FF0876FF08760308764A
:100EBD000408760B087603087601087601788C769F
:100ECD00010876FF0876FF0876FF0876FF0876FFA3
:100EDD000876030876FF0876FF0876FF0876250862
:100EED0076D00876FA0876FA0876040876FF087642
:100EFD000108760008767A0876FF087601087601F3
:100F0D00087600087603087600227887E6FFC2721D
:100F1D00BF0302D2727888E6C394036008C27DE6EF
:100F2D0030E102D27DC27E7889E630E102D27EC305
:100F3D00EF94026008758E01D273020F4F758E000B
:100F4D00C273227880E6149000809378A5F678819C
:100F5D00E6149000809378A6F67886E61490008DBE
:100F6D009378A7F67886E6F539C394025003753960
:100F7D0002789CE67538FFB402037538A0B40303FC
:100F8D0075388278A3E61490009A93F566D196226F
:100F9D00227896E6FA7897E6FB7888E6B40305C3DF
:100FAD00EB940EFB307F047A007BFFC3EB9AFCC3FE
:100FBD00948250027C827572000572EC8572F0A4E9
:100FCD00C3E5F0947D40F222D27FF19E12059B1273
:100FDD00059B7A007B007C10120591E55C2AFA7462
:100FED00003BFBDCF37C04C3EB13FBEA13FADCF7E9
:100FFD00FEC27F120F9E22757C00757D00E5EF20ED
:10100D00E6037520000520903FFFE5201460069053
:10101D001DFF1460009304600375EF1453D9BF7561
:10102D0081C043FF8012058C75EF0443B203E5B315
:10103D00240220E70DF521E5E320E0068521B343E9
:10104D00E301120E967580FF75A40075F19075D4AD
:10105D007F75903875A53F75F23F75D50075A60162
:0E106D0075E241120E96E4F8F6D8FD756801A2
:10107B00120EAB12157078988673753001C2AF12D1
:10108B0005A51205B512059B1205BC12059B120591
:10109B00C312059B12168D1205A51205A51205A0EC
:1010AB00C2AF757C00757D0078FA79FA308707D965
:1010BB00FBD8F7021C00120F17120F50120F9D12C4
:1010CB000F9E78988673120E967588107589027527
:1010DB00C82475910475D84075A82275B80275E6B9
:1010EB0090759B80759D0075D10775BC5875BB06B7
:1010FB0075BA1175E88012058CD2AF12084475369B
:10110B000053DACF207E0343DA20307E0343DA101C
:10111B0043DA01C2D8C2711205A5D2617B037A0CE6
:10112B00E55B70077A0CDB030210AB12059B20709A
:10113B00030210ABC270E55CC3940240E1E52F548F
:10114B001F855E5DF55EB55DD5DAD5C26153DACF2D
:10115B00207E0343DA20307E0343DA10C2D8C271FB
:10116B0078A2E67008D274E52F54E0F52FC275759E
:10117B0029001205A0307409C3E529940A4002D254
:10118B007512059178023074027800C3E55C9840C3
:10119B00F0C2AF1205B51205B51205B5D2AF1205E7
:1011AB00A5754C007888E6B4030241AB1205917823
:1011BB008CE6C3940150030212ABE530C39401508B
:1011CB00030212AB757CA5757DF1207435C3E55C0C
:1011DB0094FF50030212ABC2AF1205CAD2AF120575
:1011EB00A0C3E55C940150EFC2AF1205B512059692
:1011FB001205B5D2AF1205A0C3E55C94FF40E9021E
:10120B0017127F05D27F120F9E1205A0C2AFC27FAD
:10121B00120F9EAE5CC3E55C947FD2AF500241BB14
:10122B0012058CC2AF1205CAD2AFDFD8120FD5C3CD
:10123B00EE94057897F61205A51216957F0AD27FC4
:10124B00120F9E1205A0C2AFC27F120F9EAE5CC3DF
:10125B00E55C947FD2AF50E412058CC2AF1205B59A
:10126B001205961205B5D2AFDFD4120FD5EE2403BB
:10127B007896F6F87997E7C394824003985006E87E
:10128B0024827897F61205A51215B21216C4120510
:10129B00A0120F9EC3E55C94FF500221CF021712E0
:1012AB00757C00757D00C3E55C954C4003855C4CFB
:1012BB001205A078017988E7B403027805C3E55CD1
:1012CB0098400221AFC2AF1205CA1205CA1205CA55
:1012DB00D2AF1205A5753000E4F531F5320531E5D5
:1012EB0031F4703F0532789AE6781914601278322F
:1012FB0014600D787D14600878FA14600375320061
:10130B00C3E53298401D120E9612058C15327531BD
:10131B000078998673C2AF1205CAD2AF78988673DC
:10132B001205A0120596E52A700530740201AB7800
:10133B00012074027806C3E55C9840A17888E6C367
:10134B00940360031205A0E52A70030210ABC2AF31
:10135B00120E96E4F522F523F524F525F526F5670F
:10136B00D2AF7885E6C333F565E4F544F545F5462C
:10137B00F547F548F570F52CF52DF53775700875B3
:10138B00BB1012058C12084830EDFDA8BDA9BEE9B3
:10139B007001F8887112084C75700875BB10120F2C
:1013AB0017C2AF7561FF1208C28522618522628563
:1013BB002263D2AF752201752401752501752601B3
:1013CB00856069756A017888E6B40307C27D30765B
:1013DB0002D27DD268D269753300120DF0120E1F46
:1013EB001208E21208E91208E21208E91208E212E6
:1013FB000B671206AB120C5D120CA41208E9120B50
:10140B0056306E031206AC2066031207FE306603DD
:10141B0012082E120C5D120CD31208E9120B673056
:10142B006E031206E8120C5D120D4A1208E9120B3C
:10143B0056306E03120746120C5D120D791208E935
:10144B00120B67306E031207A3120C5D120DF01214
:10145B0008E9120848120B56120C5D120E1F1208E7
:0D146B004C1208E930692F856461856462C8
:10147800856069756A0179187A0CC3E53399400C5F
:10148800C269D26A8A357561FF0214A1C3E55C940A
:101498000140030213FA021527306A1D206C1AE571
:1014A80035147006C26AD26B61FAF535C3E55C94EF
:1014B8000140030213FA021527753600788279A4D1
:1014C800E760027803C3E55F985054307404E52A56
:1014D800604D7888E6B40317207D0520760781F7EC
:1014E80030760281F7206C07D26C85646181397887
:1014F800F0306C058564617820C3E541985002613D
:10150800FA306C1BC26CC27D307602D27DD26A750D
:10151800351285646161FA0536E55C6002A12A75B9
:101528003600C2AF120E967887E6FE7602120F17C3
:101538007887EEF6E4F522F523F524F525F526F56A
:1015480065752C00752D00D2AF1205A0120E967885
:10155800A4E66006D290D291D292307409C3E536DF
:101568009404400201AB41E3901A0D78201215F45F
:10157800E520B45A0CA31215F4E520B4A50302150E
:1015880092120EAB1215B20215B1901A0378807B35
:101598000A1215F4A308DBF9901A0F788C7B19123C
:1015A80015F4A308DBF9901A2822C2AF12163712D5
:1015B8001614901A00740E1215F9A374071215F96F
:1015C800A374151215F9901A0378807B0A1215F87E
:1015D800A308DBF9901A0F788C7B191215F8A30869
:1015E800DBF912164A121628901A2822E493F622DA
:1015F800E6438F01538FFDFFC3E583941C4001220E
:10160800EF857CB7857DB7F0538FFE22438F024369
:101618008F01857CB7857DB7901A0DF0538FFC221A
:10162800901A0D745AB1F9901A0E74A5B1F9227A6C
:101638003079D07820901A40B1F4E520F709A3DA80
:10164800F7227A3079D0901A40E7B1F909A3DAF98C
:1016580022AB74A875BB01027984BB02027985BBF1
:1016680003027986BB04027992BB05027987BB061F
:101678000279A3BB0702799CBB08027988BB0902DF
:101688007989E8F7227C051205A5DCFB22C2AF1296
:1016980005B51205BC1205C31205CA120596120536
:1016A800B51205BC1205C31205CA1205961205B576
:1016B8001205BC1205C31205CAD2AF22C2AF120569
:1016C800CA1205C31205BC1205B51205961205CA41
:1016D8001205C31205BC1205B51205961205CA12E9
:1016E80005C31205BC1205B5D2AF22AE74AF75C2E0
:1016F800AF1205B51205B51205B5120596DEF21240
:1017080005CA120596DFF8D2AF22D195D18DD18DB9
:10171800757401757501757600D1F37C05AD5C12A1
:1017280005A5C3ED955C70F5C3E55C9401400AC35B
:10173800E55C94FF403202174ED159B1B2D195C23F
:10174800AF75EF14D18DDCD50576C3E576940350DB
:101758000280C6D18D0575E5741490009F93F80832
:10176800C3E57598500280AED18DD18D0574C3E55F
:1017780074940A5002809C120EABB1B2C2AF75EFDE
:0317880014D18DEC
:0319FD00021004D1
:101A00000E0715FFFFFFFF03040B0301015AA50199
:101A1000FFFFFFFFFF03FFFFFF25D0FAFA04FF01DE
:091A2000007AFF0101000300FF40
:101A400023585033412320202020202020202020F4
:101A500023424C48454C4923463333302320202031
:101A60002020202020202020202020202020202076
:101C0000C2AFC2D353D9BF7581C043B20343FF8073
:101C1000752438752503B1DC7529A5752AF175E29F
:101C20004043F18053A47F75D4FFD2877DFA7803B7
:101C300079E67C10752200752300901DE97B0675FE
:101C400024987525013087028145208708D8FBD963
:101C5000F9DCF781B7308708D8FBD9F9DCF781B711
:101C6000B19CE493A3C39A6004DDC381B7DBDBB10D
:101C70008E6002812E7B08E493FAA3B16FDBF87AC1
:101C800030B16F752200752300B18EEAFCEBFDC305
:101C9000ED94FE400EB18E8A278B28ED30E0048A49
:101CA000828B83B18E7AC270D8C3ED94FE601950D6
:101CB000CEBD002BEC600F7520007521FF7529004B
:101CC000752A000200008100A827A9280809D80465
:101CD000D90281DCB192EA89AAF281CE0D81A3C337
:101CE000ED94035053EDA2E092007AC5C3E58294CF
:101CF00000E583941C508A200010438F02438F011B
:101D00008529B7852AB7F0300029A827A92808090E
:101D1000438F01538FFDD804D902A133C3E58394C7
:101D20001C4003A3A11689AAE28529B7852AB7F02A
:101D3000A3A116538FFC817F7AC1BD030CE493A34A
:101D4000FAB153DCF8B14B817F8181AA22AB23B178
:101D50006FEBFAEA6222752608C3E52313F523E543
:101D60002213F52250066323A0632201D526EAB18F
:101D7000DCB1DC75260AEAF4200102D287300102C8
:101D8000C287B1DCC3134002C201D526EB22B19257
:101D9000EAFB208702A192308702A197752608AE40
:101DA00024AF25C3EF13FFEE13FEB1E0B1DCC3EAAD
:101DB000133087024480FA30E703632201C3E5232E
:101DC00013F523E52213F52250066323A0632201B5
:101DD000D526D9E52265236523F52222AE24AF2539
:101DE0000E0FDEFEDFFCD20122424C48656C6934E6
:071DF000373163F3300601F7
:00000001FF
